:0600000000008A01122835
:080008000900483465346C3432
:100010006C346F34203477346F3472346C3464341D
:10002000213400348330831681008B1239308312DF
:1000300090006030F8004D201D288312031300301B
:10004000A0002008F000F1010A30F2000030F300B7
:100050005E20F201F301572003194B280530F00010
:100060000030F1008C200D3080200A308020E830F4
:10007000F0000330F1009E20831203132008F000EB
:10008000F1010130F2000030F300A52083120313C8
:100090007008A000212863004B28673083160313E3
:1000A00099001815981683121816981708007308E7
:1000B0007102031D08007208700208005720031C1B
:1000C0006428F001F10108000130F000F10108009E
:1000D0005720031D5E2864285720031D70286428BC
:1000E0005720031961280318642861285720031D2D
:1000F00061286428F001F1015720031D642861285C
:10010000831203130C1E822899000800700FF1035C
:10011000F10AF00071040800932000380319080068
:10012000802086208C2871088A0070088200F003E5
:10013000700FF10AF1037008710408000B110B1D18
:100140009F289720031D9E2808007208F007730857
:080150000318730AF10708000F
:00000001FF
